:020000040800F2
:10000000100C0020D5020008DD020008DF02000805
:10001000E1020008E3020008E50200080000000019
:10002000000000000000000000000000E7020008DF
:10003000E902000800000000EB0200084524000867
:10004000EF020008EF020008EF020008EF020008CC
:10005000EF020008EF020008EF020008EF020008BC
:10006000EF020008EF020008EF020008EF020008AC
:10007000EF020008EF020008EF020008EF0200089C
:10008000EF020008EF020008EF020008EF0200088C
:10009000EF020008EF020008EF020008EF0200087C
:1000A000EF020008EF020008EF020008EF0200086C
:1000B000EF020008EF020008EF020008EF0200085C
:1000C000EF020008EF020008EF020008EF0200084C
:1000D000EF020008EF020008F5260008EF02000812
:1000E000EF020008EF020008EF020008EF0200082C
:1000F000EF020008EF020008EF020008EF0200081C
:10010000EF020008EF020008EF020008EF0200080B
:10011000EF020008EF020008EF020008EF020008FB
:10012000EF020008EF020008EF020008EF020008EB
:10013000EF020008EF020008EF020008EF020008DB
:10014000EF020008EF020008EF020008EF020008CB
:10015000EF020008EF020008EF020008EF020008BB
:10016000EF020008EF020008EF020008EF020008AB
:10017000EF020008EF020008EF0200080000000094
:10018000EF020008EF02000800F002F800F092F819
:100190000AA090E8000C82448344AAF10107DA45E2
:1001A00001D100F087F8AFF2090EBAE80F0013F0A2
:1001B000010F18BFFB1A43F001031847F85700005E
:1001C00018580000103A24BF78C878C1FAD85207EE
:1001D00024BF30C830C144BF04680C6070470000C1
:1001E0000023002400250026103A28BF78C1FBD840
:1001F000520728BF30C148BF0B6070476E2900F01E
:100200009F82702900F0F783662903F040836529F7
:1002100003F03D83672903F03A83612903F03983B2
:1002200003681B0A28BF41F08001692900F04C8255
:10023000642900F04982752900F046826F2900F098
:100240008483782900F0C383E92900F01F83E4291F
:1002500000F01C83F52900F01983EF2900F0818359
:10026000F82900F0C2830368DB0928BF41F0800150
:10027000632900F0A082732900F0A582E32900F031
:10028000FB87F32901F00080002070471FB503F0C1
:10029000F9FA01F04BF804000020002103F0DCFA29
:1002A000401C60600020002103F0C0FAE0601FBD28
:1002B00010B510BD01F00CF81146FFF7E7FF03F091
:1002C000D5F801F0E9F803B4FFF7F2FF03BC01F041
:1002D00031F900000948804709480047FEE7FEE77A
:1002E000FEE7FEE7FEE7FEE7FEE7FEE7FEE7FEE7E6
:1002F00004480549054A064B704700005D24000884
:100300008901000810060020100C002010080020B1
:10031000100800201CB50C46064B7B446946009033
:10032000204600F026FA04460020694600F034FA20
:1003300020461CBD7B0400000FB41CB5084B06AA68
:100340007B4469460090059800F013FA04460020AB
:10035000694600F021FA20461CBC5DF814FB000041
:100360005504000070B50C460546012A05D02878D2
:10037000800600D5EA69002302E0012305E05B1C4A
:10038000934202D2E05C0028F9D1A869E618C01AAD
:10039000A861286A18442862284600F05BF904E046
:1003A000D5E9012114F8010B9047B442F8D328464F
:1003B00000F066F970BD00002DE9F05F8946044643
:1003C0004FF0000ADFF874B1FB44C0F820A02046CB
:1003D000E1688847002874D0252806D0D4E9012197
:1003E0009047206A401C2062F1E700265F462046C5
:1003F000E16888472028054607DB312D05D27819AA
:1004000010F8200C08B10643F1E7B00701D526F03B
:100410000406C4F81CA00027C4F818A02A2D09D08F
:10042000284602F07AFC38B304EB8708303DC8F860
:10043000185019E059F8041B204604EB870291611B
:10044000E1688847012F054618D1E069002820DAC5
:1004500026F020061DE0D8F8180000EB800005EB20
:1004600040003038C8F818002046E1688847054643
:1004700002F053FC0028EED1012F0AD02E2D08D116
:100480002046E16888477F1C0546022F46F020067B
:10049000C4DBA069002803DA404246F00106A061EF
:1004A000F00701D026F010066C2D0BD0682D09D076
:1004B0004C2D39D06A2D35D0742D35D07A2D33D0CE
:1004C00016E038E0E1682F4620468847B8420546E6
:1004D00009D16C2F26D04FF48060E1680643204696
:1004E0008847054604E06C2F1AD04FF4807006430D
:1004F0000DB3A5F14100192802D8203546F4006655
:100500004A462946204626604E46FFF777FE80B1D0
:1005100001280BD0F61D26F0070000F1080956E768
:100520004020E4E78020D8E70020D6E706F1040960
:100530004DE7284652E7206ABDE8F09FE8540000E6
:10054000421E12F8013F002BFBD111F8013B002B9A
:1005500002F8013BF9D1704710B5203AC0F00B808A
:10056000B1E81850203AA0E81850B1E81850A0E8B7
:100570001850BFF4F5AF5FEA027C24BFB1E8185011
:10058000A0E8185044BF18C918C0BDE810405FEA81
:10059000827C24BF51F8043B40F8043B08BF7047FD
:1005A000D20728BF31F8023B48BF11F8012B28BF02
:1005B00020F8023B48BF00F8012B70474FF00002C3
:1005C0000429C0F0128010F0030C00F01B80CCF165
:1005D000040CBCF1020F18BF00F8012BA8BF20F8D3
:1005E000022BA1EB0C0100F00DB85FEAC17C24BF27
:1005F00000F8012B00F8012B48BF00F8012B7047D1
:100600004FF0000200B5134694469646203922BFAB
:10061000A0E80C50A0E80C50B1F12001BFF4F7AFF6
:10062000090728BFA0E80C5048BF0CC05DF804EBD8
:10063000890028BF40F8042B08BF704748BF20F846
:10064000022B11F0804F18BF00F8012B7047704744
:100650007047704770B5044685690068C10601D5CA
:10066000302600E02026C00707D070BDD4E9012164
:1006700030469047206A401C20626D1EF6D570BD42
:1006800070B5044685690078C00707D170BDD4E90C
:10069000012120209047206A401C20626D1EF6D563
:1006A00070BD09684A0501D540B27047C905FCD53F
:1006B00000B2704709684A0501D5C0B27047C90544
:1006C000FCD580B2704700002DE9F04106460024B9
:1006D00010687529314616A510D0FFF7E2FF0028F3
:1006E00002DA404213A507E031688A0701D512A556
:1006F00002E0490704D511A5012401E0FFF7DAFF64
:1007000000210A2206F1240709E0B0FBF2FCB0FB4D
:10071000F2F302FB1C00303078541846491C0028C4
:10072000F3D123462A463046BDE8F04100F0B3B984
:10073000000000002D0000002B0000002000000041
:1007400011680268006A530501D508700AE0D305F4
:1007500001D5088006E0130603D5C217C1E90002DF
:1007600000E008600120704701694A1C02610878B6
:10077000704700B58FB0CDE90131002105910549E1
:100780007944CDE9031011466846FFF715FE0FB016
:1007900000BD0000E5FFFFFF0A6802F8010B0A60D8
:1007A000704710B5436913B1AFF3008001E0FFF764
:1007B000D9FD012010BD127800F124010A70002239
:1007C0004A700122EDE711684FF0FF32E9E70000BF
:1007D0002DE9FF5F15468A460446DFF8AC80F844F1
:1007E0000027D8E900103E46CDE9001010E03AF8A5
:1007F00016106A4602A800F04BFD411C07D0217874
:10080000890603D5E269391891420DD80744761C50
:100810002078800602D5E069B84205DDAE42E6DB0D
:100820003AF816000028E2D1A069C01BA06120465A
:10083000FFF710FFD8E90010CDE90010002017E005
:100840003AF818106A4602A800F022FDB0F1FF3F06
:1008500081460BD000250DF1080B05E0D4E90121FC
:100860001BF8050090476D1C4D45F7D308F10100BA
:10087000B0428046E4DB206A384420622046FFF71D
:10088000FFFEBDE8FF9F0000E65000002DE9F041AB
:100890008046D21D22F007020025D2E90002F52988
:1008A00015A614D0011E72F1000106DA0023D0EB68
:1008B000030063EB020211A608E0D8F800108B07D2
:1008C00001D50FA602E0490701D50EA60125114664
:1008D000002408F1240704E000F098F830323A557B
:1008E000641C50EA0102F7D12B46324621464046AD
:1008F000BDE8F04100F0CFB8000000002D0000007E
:100900002B0000002000000030B4002100F124047E
:1009100008E002F00705D208303542EA4372DB08EE
:100920006554491C52EA0305F3D10468002310A260
:10093000250707D5A40600D421B1C46901230DA25F
:10094000641EC46130BC00F0A6B810B50446214650
:100950001068FFF7AFFE02462046BDE810400023B6
:10096000D2E7D21D22F00701D1E90023CCE7000035
:100970000000000030000000F0B40D4601880905B9
:1009800002D5214C7C4402E01F4C7C440E340021F3
:1009900000F1240608E002F00F071209E75D42EAC1
:1009A00003721B097754491C52EA0307F3D10278FA
:1009B0000023120704D5702D06D009B1022311348B
:1009C0002246F0BC00F067B801231034F8E770B598
:1009D00004460D4621461068FFF76CFE0246294684
:1009E0002046BDE870400023C6E7D21D22F0070371
:1009F000D3E90023C0E70368126843F020030360D3
:100A00000823C3610023B7E7484F000030B5B0F1B9
:100A10000A024FEA900E71F100034EEA817EB0EBBC
:100A20000E0061EB91014FEA101E4EEA017E10EBC1
:100A30000E0041EB11114FEA102E4EEA016E10EB41
:100A40000E0041EB11214FEA104E4EEA014E10EB21
:100A50000E0041EB1141401841F100014FEAD00076
:100A600040EA41704FEAD10110EB80054FEA810462
:100A700044EA907444EB01046D1944EB0404521BE6
:100A8000A3414FF0000348BF0A3200D530BD401CDF
:100A900041F1000130BD2DE9F0470D4699469246DF
:100AA000044600F124080168880604D5E06921F0B5
:100AB0001001216000E00120A84201DD471B00E099
:100AC0000027A1697A1902EB0900081AA0612078B1
:100AD000C00602D42046FFF7BDFD002608E0D4E999
:100AE00001211AF806009047206A401C761C2062FB
:100AF0004E45F4DB2078C0060AD52046FFF7AAFD54
:100B000006E0D4E9012130209047206A401C206291
:100B1000381EA7F10107F4DC07E0D4E9012118F839
:100B200005009047206A401C2062281EA5F101059F
:100B3000F3DC2046FFF7A4FD2078000602D5022052
:100B4000BDE8F0870120FBE770472DE9FF4F0C4619
:100B50001E464FF0FF378BB0D2E90001DDF8608010
:100B60000A908A46C1F30A5505B93D460021084658
:100B70004FF00000BAF1000F00F4400005DA00EB7E
:100B800080004FF4400101EA50004FEA9059B9F15A
:100B9000010F00DDB9460A9850EA4A000ED044F62B
:100BA0001050A5F2FF3545432F14B8F1000F1ED0A9
:100BB0007542291E1EDDC9F100021CE0B8F1010FCB
:100BC0004FF0000001D0302103E0F24305E0215452
:100BD000401CB042FBDB30460022002121540B991F
:100BE000C1F80880C1E900200FB0BDE8F08FBD1B3F
:100BF0006D1CDEE74A4600DA694206A800F0DAFB1F
:100C000006AB93E8070003AB83E8070050460A9958
:100C100000F097FC8DE80700A0F500501F38009009
:100C20000398002D0ADD42F21F014A4608440023C2
:100C300003A90390684600F000FF09E0A0F500500A
:100C40004A461F38002303A90390684600F00AFFB4
:100C50008DE807000004000C03D04FF0FF3041087E
:100C600000E01046B8F1000F03D0002200921546B4
:100C70001EE0751E05D4FFF7C9FE303262556D1EA9
:100C8000F9D5B3460122084302D000227F1C04E0BC
:100C90002078302801D100227F1E002A099784D0B5
:100CA0001DE0112D07DAFFF7B1FE303262556D1CE1
:100CB00050EA0102F5D1084302D00098C8B10EE015
:100CC0000021681E05E0235C625C63542254401ED0
:100CD000491C8142F7DBAB46A81B401E099000204F
:100CE00004F80B000B98099AC0F80880C0E9002BA3
:100CF0007AE711264FF0000857E72DE9F04F8846B4
:100D00000446D21D22F0070191B0D1E90001CDE9DE
:100D10000A0101F0EAFF02460B98C00F01D02D2016
:100D200007E02068810701D52B2002E0202101EA9D
:100D3000C000032A099001D0072A05DB034641467B
:100D4000204600F0F7FA0BE12078800601D5E06933
:100D500000E00620B8F1650F814606D0B8F1660FB5
:100D600018D0B8F1670F70D131E00020B9F1110F40
:100D7000009001DB112301E009F101030AAA01A996
:100D80000CA8FFF7E2FEDDE90C70002609F1010571
:100D9000834647E001204B4600904FF000470AAAE7
:100DA00001A90CA8FFF7D1FEDDE90DB00C995D4655
:100DB000002610B909F101000D18B9EB050003D4A4
:100DC000C0F1FF3609F10105A5EB09002BE0B9F1EF
:100DD000010F01DA4FF001090020B9F1110F009065
:100DE000484601DD112300E003460AAA01A90CA828
:100DF000FFF7ABFEDDE90C704D46002683462078F8
:100E000000070AD4AB4500DA5D4601A8012D04DDD8
:100E1000411911F8011C302907D04F4502DA17F1AA
:100E2000040F04DA012082460FE06D1EEEE7002F6A
:100E300002DCED1B3E4403E0781CA84200DD7D1C73
:100E4000B81B00F1010A4FF000472078000703D4D7
:100E5000AA4501DB4FF0FF3A0021B7F1004F0DF139
:100E600043088DF8431024D002202B23002F01DAF1
:100E70007F422D230A21021EA0F1010000DC5FB198
:100E800097FBF1FC97FBF1F201FB1C7C17460CF180
:100E9000300C08F801CDEEE7A8F1010003702188BD
:100EA000090501D5452100E06521A0F1010800F800
:100EB000011C09980FA9A1EB0807FF1D00B1012033
:100EC000411901EBEA70A1693844081A401EA0617B
:100ED0002078C00602D42046FFF7BCFB099828B151
:100EE000D4E901219047206A401C20622078C00686
:100EF00022D52046FFF7AEFB1EE0002E04DBB345F3
:100F000002DD01A8805D00E03020D4E90121904796
:100F1000206A401C2062761CAAF101005FEA000AE8
:100F20000AD100F003FAC0680168405CD4E90121ED
:100F30009047206A401C2062281EA5F10105DCDCD8
:100F400007E0D4E9012118F8010B9047206A401C02
:100F50002062381EA7F10107F3DC2046FFF790FB63
:100F6000032011B041E600002DE9F04F04460D4684
:100F7000D21D22F0070089B0D0E9009748463946D3
:100F800001F0B3FE0246F80F01D02D2307E02068E0
:100F9000810701D52B2302E0202101EAC0038DF84F
:100FA00020300BB1012000E00020032A824601D04E
:100FB000072A04DB2946204600F0BCF93FE12078EF
:100FC000800601D40D2500E0E569C7F30A560D2D12
:100FD00049DA00214FEA175B08464FF00000002F66
:100FE00000F4400007DA00EB80004FF4400100EB12
:100FF000D07001EA60008115012901DD4FF0FF3159
:1010000000224FEA850CBCF1180F06D31346ACF151
:1010100018004FF08052C24003E04FF4801323FACF
:101020000CF30CF10C0CBCF1200F04D3ACF1200C30
:1010300009FA0CF001E007FA0CF000294FF0004823
:1010400001DD18B90FE00ED140450CD319EB0209B0
:101050005F4121B9404502D19F4329EA0209BBEB18
:10106000175F00D0761C2088000502D57B487844A5
:1010700002E07A487844193808AA302302F80A3086
:10108000037C0AF10101002E0AF1020A53546A4658
:1010900002DC4FF0300101E04FF031014FF0010868
:1010A0008DF8001002D0A6F2FF3603E059EA47019E
:1010B00000D06B4E002D02DC2178090704D54FF0DB
:1010C00002082E218DF80110C44600210BE0C7F361
:1010D00003433F01C35C491C6D1E02F8083005291B
:1010E00008F1010801DA002DF1DC00210CE000EB31
:1010F0001973491C1B786D1E082902F808304FEA45
:10110000091908F1010801DA002DF0DC21688B06CD
:1011100002D516E0A8F10108E04505DD02EB080361
:1011200013F8013C302BF5D0B8F1000F09DD02EBCC
:10113000080313F8013C2E2B03D1090701D4A8F1B1
:101140000108002D05DD3E2102F808106D1E08F192
:101150000108407C002E02F8080008F1010804DABA
:101160002D20764202F8080002E02B2002F8080049
:101170000A214FF47A70864208F101080BDB96FBD6
:10118000F0F3303302F8083096FBF0F308F1010871
:1011900000FB136601E0642E0CDB642096FBF0F389
:1011A000303302F8083096FBF0F308F1010800FB39
:1011B000136601E00A2E06DB96FBF1F0303002F8F0
:1011C000080008F1010896FBF1F001FB10603030D7
:1011D00002F80800A16908F1010808EB050202EB1A
:1011E0000A00081AA0612078C00602D42046FFF742
:1011F00031FA216A08AE01EB0A00206204E0D4E96A
:10120000012116F8010B9047BAF1010AF7D22078B4
:10121000C00602D52046FFF71DFA6E4609E016F813
:10122000010B3E280FD0D4E901219047206A401CD1
:101230002062B8F10108F2D22046FFF721FA09B086
:101240000320BDE8F08F206A2844206203E0D4E93F
:101250000121302090476D1EEBD3F8E7994800003C
:1012600002FCFFFF10B5436913B1AFF3008001E04A
:10127000FFF7AEFA012010BD128800F1240182842C
:101280000022C2840122EDE711684FF0FF32E9E746
:1012900070B516460C46054600F040F8036893F812
:1012A0000101012806D0FF2C0FD8185D68B101207C
:1012B0002C7070BDD3F807013246214603F20713A4
:1012C00003442846BDE8704018474FF0FF3070BD1A
:1012D000754600F0EBF8AE4605006946534620F02F
:1012E0000700854618B020B5FFF702F8BDE820409A
:1012F0004FF000064FF000074FF000084FF0000BD2
:1013000021F00701AC46ACE8C009ACE8C009ACE884
:10131000C009ACE8C0098D467047000010B500F068
:1013200005F8001D10BD00BF3125000000487047C2
:10133000CC0500202DE9F0411F4604460326016834
:10134000072A01F4006004DB08B116A505E016A524
:1013500003E008B115A500E015A521F010002060FC
:10136000A069C01EA0610FB1401EA0612046FFF71A
:1013700071F94FB1D4E9012138469047206A401CE9
:101380002062C01C206206E0206AFAE7D4E901214D
:1013900015F8010B9047761EF8D22046FFF770F93A
:1013A000BDE8F0814E414E006E616E00494E460030
:1013B000696E66002DE9F047814616468AB03548C9
:1013C00078440DC88DE80D0032487844801C03AC89
:1013D0000DC884E80D0041F69B300844372190FB8E
:1013E000F1F290FBF1F5A5F1800501FB12041B3C25
:1013F00002D56442012000E00020DFF898A080467A
:101400000027FA44AAF1BE0A0EE0E0070AD03246ED
:10141000684607EB470101230AEB810100F022FB3C
:101420008DE8070064107F1C002CEED1194F7F441B
:10143000AE3F19E0E80715D007EB04100DF1180ACC
:1014400090E80E008AE80E00C068F04201D19819B9
:1014500008903246012306A903A800F003FB03AB62
:1014600083E807006D10641C002DE3D14FF00103E9
:1014700032466946B8F1000F03A802D000F0DDFA49
:1014800001E000F0EFFAC9E90001C9F808200AB04C
:10149000BDE8F087D845000010B50446AFF30080E2
:1014A0002046BDE81040FEF70EBF00000048704720
:1014B000AC0500204FF0013C50F8042B51F8043BE0
:1014C0009A4221D1A2EB0C03934313EACC1317D118
:1014D00050F8042B51F8043B9A4215D1A2EB0C03AF
:1014E000934313EACC130BD150F8042B51F8043B6F
:1014F0009A4209D1A2EB0C03934313EACC13DBD03D
:101500004FF00000704700BFD01A01BAB1FA81F164
:1015100001F0180122FA01F0CB40C1F12001DBB249
:10152000C0B2C01A2CFA01F3D11A914311EAC311C7
:10153000E6D1704701491820ABBEFEE72600020045
:1015400070475FEA400C08BF91F0000F4FEA8C2310
:101550004FEAC12243EA51514FEA1C5018BF00F52F
:10156000F0404FEA300018BF41F000415FEA6C5C88
:1015700000F02980BCF1FF3F08BF40F08040704779
:10158000130C06BF12044FF0100C4FF0000C130E9A
:1015900004BF12020CF1080C130F04BF12010CF16E
:1015A000040C930F04BF92000CF1020CD30F04BF84
:1015B00052000CF1010C11464FF00002A0F11F0087
:1015C000A0EB0C00704711F0004F08BF704731F0DE
:1015D00000413FF4D5AF0B0C06BF09044FF0100CCF
:1015E0004FF0000C0B0E04BF09020CF1080C0B0F9E
:1015F00004BF09010CF1040C8B0F04BF89000CF12E
:10160000020CCB0F04BF49000CF1010CCCF12003FC
:10161000A0EB0C0022FA03F302FA0CF241EA0301F8
:1016200000F10100704720F07F4C80EA030023F0B6
:101630007F47ACEB070303F57C5300F0004003F158
:10164000FF032DE980494FEA154B09B44FEA1443D3
:1016500025EA0B4E24EA03480FF2042606EB132773
:1016600049083E785FEA320203FB0667C7F50007C8
:1016700007FB06F64FEA54374FEAD64606F1020654
:1016800007FB066CCCF1005C4FEA1C472CEA074CC8
:1016900007FB06F40CFB06F504EB15464FEA96161D
:1016A00034BF00204FF000404FEAD13706FB07FC63
:1016B0004FEA1C4C0CFB0BF7D21B03FB0CF761EB46
:1016C00007010CFB0EF7B0EB074072EB17420CFB67
:1016D00008F734BFA2EB0742B2EB074261EB1741B8
:1016E0004FEA0C444FEA910706FB07FC4FEA1C4CFB
:1016F0000CFB0BF7B0EBC74072EB573203FB0CF758
:1017000034BFA2EBC742B2EBC74261EB57310CFBCF
:101710000EF7B0EBC70072EB57720CFB08F734BF43
:10172000A2EBC702B2EBC70261EB5771039F4FEA0E
:10173000816141EA921104EBCC044FEAD1374FEAC0
:10174000826206FB07FC42EA90124FEA80604FEA91
:101750001C4C0CFB0BF7D21B03FB0CF761EB0701D6
:101760000CFB0EF7B0EB074072EB17420CFB08F7CF
:1017700034BFA2EB0742B2EB074261EB17414FEADD
:101780008C554FEA910704EB9C2406FB07FC4FEABB
:101790001C4C0CFB0BF7B0EBC74072EB573203FB52
:1017A0000CF734BFA2EBC742B2EBC74261EB573133
:1017B0000CFB0EF7B0EBC70072EB57720CFB08F78F
:1017C00034BFA2EBC702B2EBC70261EB577115EB56
:1017D0004C254FEA816141EA92114FEA82624FEA59
:1017E000D13742EA901206FB07FC44F100044FEAAD
:1017F00080604FEA1C4C0CFB0BF7D21B03FB0CF771
:1018000061EB07010CFB0EF7B0EB074072EB1742E0
:101810000CFB08F734BFA2EB0742B2EB074261EBC7
:10182000174115EB1C154FEA813141EA92414FEA0D
:10183000823242EA90424FEA80304FEA0C7644F11D
:10184000000448EA03434EEA0B484FF0000EB2EBA7
:10185000080C71EB030724BF624639464EEB0E0EAF
:101860004FF0000B0018524149414BEB0B0BB2EB10
:10187000080C71EB03077BF1000B24BF624639466D
:101880004EEB0E0E4FF0000B0018524149414BEB4E
:101890000B0BB2EB080C71EB03077BF1000B24BFC1
:1018A000624639464EEB0E0E51EA020718BF46F06B
:1018B000010616EB0E7655F1000254F1000103D536
:1018C000BDE88901BDE80088BDE88901BDE80048A0
:1018D000B619524141EB0101A3F101037047808029
:1018E0007F7E7D7C7B7A797877767675747372717A
:1018F00071706F6E6E6D6C6C6B6A6A696868676632
:1019000066656464636362616160605F5F5E5E5DC3
:101910005D5C5C5B5B5A5A59595858575756565537
:1019200055555454535352525251515050504F4F99
:101930004F4E4E4D4D4D4C4C4C4B4B4B4A4A4A49E9
:10194000494948484847474747464646454545442C
:101950004444444343434342424242414141002BB9
:101960009C4630D477002BD01CB54FEA370703B420
:101970004FF010004FF01001BAF1000F06D0BCF18B
:10198000000FDCBF40F0080040F008014FF00000FD
:101990000FBCBDE810400BF1010BBBF1010F08BFFC
:1019A0005FEA170722BF12F1010211F101014FF0A6
:1019B000004143F1000300F0004043EA000070479B
:1019C000F9D35708D0E746EA064613F1400F4FEA2D
:1019D00016461FDD13F1200FDFBF16430A46002114
:1019E00020335B42BED0C3F1200746EA064602FA26
:1019F00007F74FEA164646EA0706C3F1200722FA20
:101A000003F201FA07F721FA03F14FF0000342EA6B
:101A10000702A7E746EA020646EA06464FEA1646E6
:101A200046EA0106BCBF46EA0646360C4FF0000304
:101A30004FF000024FF0000194E72DE9804C9A46E8
:101A4000934670B491E8380007C831EA400C48BFAB
:101A500034EA430C03D5FFF7E6FDFFF780FFF0BC47
:101A6000BDE8008C2DE9804C9A46934670B491E80D
:101A7000380007C810F0804F08BF13F0804F03D123
:101A800000F005F8FFF76BFFF0BCBDE8008C20F01C
:101A90007F4780EA030023F07F4C07EB0C03A3F59C
:101AA0007C5300F00040A3F1FE0392F0000F00F021
:101AB000B38095F0000F00F077802DE901494FEADF
:101AC00011404FEA144621EA004800FB06FC24EAD4
:101AD000064708FB06F607FB08F800FB07F718EBBC
:101AE00006484CEB164C4FEA124B18EB07484FEAEE
:101AF00015464CEB174022EA0B4E0BFB06FC25EA81
:101B000006470EFB06F607FB0EFE0BFB07F71EEB68
:101B1000064E4CEB164C4FF000061EEB074E4CEBFE
:101B2000174B18EB0B0840F1000018EB0E0B58EBAD
:101B3000000840F100008F1A4FF000013CBFC9437C
:101B4000661B14BFB5EB040C00213CBFC943F61B58
:101B50004FEA17444EEA8E0E27EA04454FEA1C4727
:101B600004FB07622CEA074C05FB07F70CFB05F6A4
:101B700004FB0CFC16EB074642EB174216EB0C4637
:101B800042EB1C421BEB060658EB0202414146EABF
:101B90009E0601D5BDE80189B619524141EB01010C
:101BA000A3F10103BDE801894FEA14454FEA11474B
:101BB00024EA054621EA074C05FB07F406FB07F774
:101BC0000CFB06F105FB0CFC11EB074144EB174441
:101BD0004FEA124711EB0C4144EB1C4422EA074C3C
:101BE00005FB07F206FB07F70CFB06F605FB0CFCF2
:101BF00016EB074642EB174216EB0C4642EB1C4530
:101C00006A1854F1000148BF7047B619524141EBC0
:101C10000101A3F10103704795F0000F37D04FEA9F
:101C200011424FEA144721EA024624EA074C02FB1C
:101C300007F106FB07F70CFB06F402FB0CFC14EBA8
:101C4000074441EB17414FEA154714EB0C4441EBB5
:101C50001C4125EA074C02FB07F506FB07F70CFBC6
:101C600006F602FB0CFC16EB074645EB174516EB98
:101C70000C4645EB1C42121951F1000148BF704758
:101C8000B619524141EB0101A3F1010370474FEA3C
:101C900014454FEA114724EA054621EA074C05FBA3
:101CA00007F106FB07F70CFB06F24FF0000605FBF9
:101CB0000CFC12EB074241EB174112EB0C4251EBCB
:101CC0001C4148BF7047921841EB0101A3F1010389
:101CD0007047000051B18200A2F1C042126842F088
:101CE00001038200A2F1C042136009E08200A2F168
:101CF000C0421268034B1A408300A3F1C0431A602C
:101D000070470000FEFF0F0030B5002100220023C5
:101D10000468A400A4F1C0442168424C2140D0E9E9
:101D200001452C43C5682C4305692C4345692C4368
:101D300085692C43C5692C43056A2C43456A2C43AD
:101D4000856A2C43C56A2C43056B2C4321430468E8
:101D5000A400A4F1C04421608468082C0BD104685D
:101D6000A400A4F1C044246844F040050468A40021
:101D7000A4F1C04425600468641CA400A4F1C0441C
:101D8000226802F04042446B2468456B6D6844EA67
:101D90000514456BAD6844EA0524456BAD8944EAFA
:101DA0000544456B2D8A44EA0554456B2D7D44EA74
:101DB0000564456BAD692C4322430468641CA40090
:101DC000A4F1C0442260C46AB4F5804F20D10468F5
:101DD000A400A4F1C044D4F80431134C2340846B14
:101DE0002468856B6D6844EA0514856BAD6844EA28
:101DF0000524856BAD8944EA0544856BAD692C43A8
:101E000023430468A400A4F1C044C4F8043107E0EB
:101E10006FF070450468A400A4F1C044C4F80451F4
:101E200030BD00008000F7FF0000F0CFF0B50A469B
:101E300000210023002400BF3DE0012505FA01F345
:101E4000156805EA03049C4234D105684F00032657
:101E5000BE40B543056015794E00B5400668354370
:101E600005601579012D02D01579022D16D18568EE
:101E70004F000326BE40B543856055794E00B540FE
:101E8000866835438560456801268E40B5434560C8
:101E9000456896798E40B6B235434560C5684F00B7
:101EA0000326BE40B543C560D5794E00B540C6682F
:101EB0003543C560491C1029BFD3F0BDF0B50023E0
:101EC00000244D07ED0E02FA05F3CE1000F12005B7
:101ED00055F826504E07F70E0F26BE40B543CF10DB
:101EE00000F1200646F82750CE1000F1200555F8E5
:101EF000265045EA0304CE1000F1200545F826409F
:101F0000F0BD418370470183704700001CB501217B
:101F1000022000F07DF90121084600F079F9032044
:101F2000009002208DF8050001208DF8040069461C
:101F30001848FFF77BFF4020009003208DF8050034
:101F400001208DF804008DF807008DF80600124876
:101F5000406980F040001049486169460E48FFF72B
:101F600065FF8020009003208DF8050001208DF88A
:101F700004008DF8060000208DF80700064840692F
:101F800080F080000449486169460348FFF74EFF2E
:101F90001CBD0000000402400000024010B500F02B
:101FA00003F800F095F810BD1CB50121182000F0D1
:101FB0002FF94EF2B370009002208DF80400032038
:101FC0008DF8050000208DF8060001208DF807002F
:101FD00069463D48FFF72AFF0C2204213A48FFF7E3
:101FE0006DFF0C2205213848FFF768FF0C220721FE
:101FF0003548FFF763FF0C2208213348FFF75EFFE7
:102000000C2209213048FFF759FF0C220A212E48E3
:10201000FFF754FF0C220D212B48FFF74FFF0C2236
:1020200001212948FFF74AFF0C2200212648FFF72B
:1020300045FF0C220F212448FFF740FF0C220E2100
:102040002148FFF73BFF4FF68070009002208DF88B
:10205000040003208DF8050000208DF80600012003
:102060008DF8070069461948FFF7E0FE0C220721AA
:102070001648FFF723FF0C2208211448FFF71EFF24
:102080000C2209211148FFF719FF0C220A210F48E1
:10209000FFF714FF0C220B210C48FFF70FFF0C2257
:1020A00011460A48FFF70AFF0C220D210748FFF7E7
:1020B00005FF0C220E210548FFF700FF0C220F211F
:1020C0000248FFF7FBFE1CBD000C0240001002405E
:1020D00000B59DB00121084600F0AAF80220079043
:1020E000002008900520099000200A900B900C9089
:1020F0004FF080500D9003200090002001900620AA
:10210000029000200390012004900020059006908A
:102110000E900F90109010201190002012901390AC
:102120001490159016904FF480501790002018903E
:102130004FF48040199000201A9007A81B90CDF80A
:1021400070D00EA8FFF7E0FD01210020FFF7C2FDCF
:102150001DB000BD70B58AB004462646012102209C
:1021600000F076F80121022000F052F802200090E1
:102170008DF8040003208DF8050000208DF806007E
:102180008DF8070069461E48FFF750FE0222012124
:102190001B48FFF793FE1B4800681B49B0FBF1F09A
:1021A000401E85B264200890ADF81C500020ADF8A8
:1021B0002400ADF81E0007A9144800F0F5F96020CE
:1021C000ADF808000120ADF80A0004960220ADF831
:1021D000140002A90D4800F09DF908210B4800F0F9
:1021E000D5F90121094800F06DF90121074800F0F7
:1021F00075F90121054800F07DF90AB070BD0000B5
:102200000004024050000020A086010000040040AD
:1022100029B1064A12680243044B1A6004E0034ADB
:1022200012688243014B1A60704700003038024048
:1022300029B1064A12680243044B1A6004E0034ABB
:1022400012688243014B1A60704700003838024020
:1022500029B1064A12680243044B1A6004E0034A9B
:1022600012688243014B1A607047000040380240F8
:10227000F0B5002100220024022500260223324F5F
:102280003F6807F00C0121B1042905D0082937D196
:1022900005E02E4F076036E02D4F076033E02A4FF0
:1022A0003F1F3F68C7F38056274F3F1F3F6807F027
:1022B0003F036EB1264FB7FBF3F7DFF88CC0ACF1EC
:1022C000040CDCF800C0CCF3881C07FB0CF40CE019
:1022D0001E4FB7FBF3F7DFF870C0ACF1040CDCF86D
:1022E00000C0CCF3881C07FB0CF4174F3F1F3F685E
:1022F000C7F301477F1C7D00B4FBF5F7076002E0E0
:10230000124F076000BF00BF0F4F3F6807F0F0019A
:102310000909104F7A5C0768D74047600A4F3F6849
:1023200007F4E051890A0B4F7A5C4768D740876011
:10233000054F3F6807F46041490B064F7A5C4768D8
:10234000D740C760F0BD0000083802400024F40008
:1023500000127A00010000200CB5002001900090CE
:102360003448006840F480303249086000BF31488A
:10237000006800F4003000900198401C0190009823
:1023800018B90198B0F5A04FF1D12A48006800F4BF
:10239000003010B10120009001E000200090009872
:1023A000012846D123484030006840F08050214940
:1023B000403108602048006840F440401E490860F1
:1023C0001C48083000681B4908310860084600684E
:1023D00040F4004008600846006840F4A0500860DF
:1023E0001648091F0860081F006840F08070091F28
:1023F000086000BF0F48006800F000700028F9D0A6
:1024000040F205700E4908600A480830006820F064
:1024100003000849083108600846006840F00200DF
:10242000086000BF03480830006800F00C0008286E
:10243000F8D10CBD0038024000700040085440083C
:10244000003C024004480088002804DD024800885F
:10245000401E0149088070474E00002010B5154805
:10246000006840F47000134908601348006840F0A9
:1024700001001149086000200F49083108600E482A
:1024800000680E4908400C4908600D48091D0860A5
:10249000081F006820F48020091F086000200649FA
:1024A0000C310860FFF758FF4FF000600149803998
:1024B000086010BD88ED00E000380240FFFFF6FE26
:1024C0001030002421B1028842F08002028004E032
:1024D00002884FF67F731A400280704721B102884C
:1024E00042F00102028004E002884FF6FE731A40B7
:1024F0000280704731B1B0F8442042F40042A0F8A5
:10250000442005E0B0F84420C2F30E02A0F84420B5
:102510007047000070B5002200230024058C4EF6A1
:10252000FF7635400584038C8488828B48F6FF75DE
:102530002A404FF6FF452A400D884FF6FF7606EAFF
:1025400005252A434DF6FF752B408D8906EA053592
:102550002B434D8806EA05352B430A4DA84202D08D
:10256000094DA84208D14BF6FF752C400D8A4FF655
:10257000FF7606EA85152C43848082838D68056486
:10258000038470BD00000140000401400A460021A0
:10259000818B4FF2FF7319404FF6FF7303EA02235A
:1025A000194381837047000000220288184B98422B
:1025B0000ED0184B98420BD0B0F1804F08D0164B7C
:1025C000984205D0154B984202D0154B984204D141
:1025D0004FF68F731A404B881A43124B984207D01C
:1025E000114B984204D04FF6FF431A400B891A430F
:1025F00002804B68C3620B880385054B984202D06A
:10260000044B984201D18B7A038601238382704761
:1026100000000140000401400004004000080040A8
:10262000000C0040001000400014004000B587B0CE
:1026300001210846FFF7ECFD01214804FFF708FEE1
:10264000072203212948FFF739FC072202212748E6
:10265000FFF734FC00208DF81A0001208DF81B00D4
:1026600002208DF818000420059002208DF8190032
:1026700005A91E48FFF7DAFB02208DF81800082094
:10268000059005A91948FFF7D1FB4FF4614001906F
:102690000020ADF80800ADF80A00ADF80C00ADF868
:1026A00010000C20ADF80E0001A9114800F0AAFAA4
:1026B000262000280DDB00BF00BF00F01F02012113
:1026C00091404209920002F1E022C2F8001100BFDD
:1026D00000BF00BF012240F22551054800F06CFA0E
:1026E0000121034800F032FA07B000BD00000240AB
:1026F0000044004008B540F22551FE4800F032FA8F
:1027000000287DD0FB4800F0E7FAC0B20090FA48FC
:102710000078012875D1F9480078A8B99DF8000023
:102720000D2806D1684601F04FF80120F3490870E2
:102730000AE09DF80000F249F24A12788854F14804
:102740000078401CEF490870EC480078012815D14A
:102750009DF800000D2806D1684601F035F80220EA
:10276000E64908700AE09DF80000E549E54A12785C
:102770008854E4480078401CE2490870DF4800783B
:10278000022815D19DF800000A2806D1684601F0FC
:102790001BF80320D94908700AE09DF80010D848BA
:1027A000D84A12788154D7480078401CD54908701F
:1027B000D2480078032815D19DF800000D2806D1D5
:1027C000684601F001F80420CC4908700AE09DF841
:1027D0000010CB48CB4A12788154CA480078401C7C
:1027E000C8490870C5480078042827D19DF8000022
:1027F0000A2818D19DF80000C149C24A127801E0A8
:102800008CE11BE088540020BE490870684600F047
:10281000DBFF4021BC48FFF774FB0020B74908707C
:10282000B54908700AE09DF80000B549B54A12782C
:102830008854B4480078401CB2490870AE4800780B
:10284000022875D1AD480078A8B99DF800000D2880
:1028500006D1684600F0B8FF0120A84908700AE0D8
:102860009DF80000A649A74A12788854A548007828
:10287000401CA4490870A1480078012815D19DF892
:1028800000000A2806D1684600F09EFF02209B49FE
:1028900008700AE09DF8000099499A4A1278885415
:1028A00098480078401C974908709448007802289E
:1028B00015D19DF800000D2806D1684600F084FF70
:1028C00003208E4908700AE09DF800008C498D4A6B
:1028D000127888548B480078401C8A4908708748D1
:1028E0000078032815D19DF800000A2806D1684613
:1028F00000F06AFF0420814908700AE09DF800108A
:102900007F48804A127881547E480078401C7D4977
:1029100008707A480078042816D19DF800000D2828
:1029200007D1684600F050FF0520744908700BE09D
:1029300027E09DF800107248724A1278815471485D
:102940000078401C6F4908706C480078052824D135
:102950009DF800000A2815D19DF800106848694AC2
:1029600012788154002067490870684600F02CFFF7
:1029700040216548FFF7C5FA0020604908705E49AC
:1029800008700AE09DF800105D485E4A1278815494
:102990005C480078401C5B49087057480078032861
:1029A00075D156480078A8B99DF800000D2806D1C9
:1029B000684600F009FF0120504908700AE09DF8C0
:1029C00000004F494F4A127888544E480078401C06
:1029D0004C49087049480078012815D19DF800003D
:1029E0000A2806D1684600F0EFFE0220434908702D
:1029F0000AE09DF800104248424A1278815441484A
:102A00000078401C3F4908703C480078022815D1E6
:102A10009DF800000D2806D1684600F0D5FE032081
:102A2000364908700AE09DF800103548354A12789A
:102A3000815434480078401C324908702F4800788F
:102A4000032824D19DF800000A2815D19DF8001014
:102A50002B482C4A1278815400202A490870684675
:102A600000F0B2FE40212848FFF74BFA002023492E
:102A70000870214908700AE09DF800102048214A9A
:102A8000127881541F480078401C1E4908701A486B
:102A9000007804284ED119480078A8B99DF80000A4
:102AA0000D2806D1684600F08FFE012013490870FA
:102AB0000AE09DF800101248124A12788154114819
:102AC0000078401C0F4908700C480078012831D16B
:102AD0009DF800000A2822D19DF800000849094A03
:102AE00012788854002007490870684600F06CFE90
:102AF00040210BE000440040000000204D00002079
:102B0000340400204C000020000002400A48FFF777
:102B1000F8F9002009490870094908700AE09DF891
:102B200000000849084A1278885407480078401C79
:102B30000549087008BD0000000002404D0000205B
:102B400000000020340400204C00002021B18289C4
:102B500042F40052828104E082894DF6FF731A40EC
:102B60008281704770B502460024002300250020B2
:102B700040F66A16B14200D100BFC1F3421501F020
:102B80001F03012606FA03F3012D02D19689334073
:102B900006E0022D02D1168A334001E0968A3340C6
:102BA0000C12012606FA04F41688344013B10CB155
:102BB000012000E0002070BDF0B50346002400268F
:102BC0000025002040F66A17B94200D100BF184620
:102BD000C1F3421401F01F06012707FA06F5012C84
:102BE00001D10C3004E0022C01D1103000E014308F
:102BF0001AB107682F43076002E00768AF43076018
:102C0000F0BD00002DE9FF4705460E460024A14611
:102C100000BFA046B08900B100BF2C8A24F4405404
:102C2000F08804432C82AC8941F20C608443B08864
:102C300031890843718908430443AC81AC8A24F488
:102C40004074B0890443AC826846FFF711FB20480A
:102C5000854202D01F48854202D1DDF80C9001E088
:102C6000DDF80890A88900F4004040B109EBC900E4
:102C700000EB091031684900B0FBF1F707E009EB00
:102C8000C90000EB091031688900B0FBF1F764203E
:102C9000B7FBF0F004012009642101FB1078A8893A
:102CA00000F4004040B1322000EBC800B0FBF1F06E
:102CB00000F00700044308E0322000EB0810642114
:102CC000B0FBF1F000F00F0004432C81BDE8FF875A
:102CD000001001400014014001468888C0F308003C
:102CE0007047C1F308028280704703B40198410025
:102CF000009850EAC12018BF04204A0D18BF40F0C8
:102D0000010040F2FF72B2EB515F08BF40F00200D9
:102D1000012808BF052002B0704730380A2801D2C8
:102D200001207047002070471CB501211020FFF7DB
:102D30006FFA0820009000208DF804008DF805003F
:102D400001208DF8070069460848FFF76FF810204A
:102D5000009000208DF804008DF8050001208DF80A
:102D6000070069460148FFF761F81CBD00100240EA
:102D7000104A12684FF47A73B2FBF3F202FB00F1CF
:102D80000D4A126842F080720B4B1A6000220B4B06
:102D90005A601A46126842F001021A6000BF074AE0
:102DA00052688A42FBD3054A126822F00102034BA3
:102DB0001A60704750000020FCED00E0001000E0B9
:102DC000F0B50446DDE9055600200EB140F00400E0
:102DD0000DB140F008000BB140F010000AB140F016
:102DE000200009B140F040000CB140F08000F0BD7F
:102DF0002DE9FF4F81B004460D469A4639480088B8
:102E0000A0420FDD37484088A8420BDD3648806875
:102E100080882044002805DB33488068C088284427
:102E2000002802DA05B0BDE8F08F2F498968C8880C
:102E3000C11700EB5171C1F3C7074FF0000800261E
:102E400048E04FF0000B3FE003982038264989689E
:102E5000C9884843784306FB0700584422498968DB
:102E60000968085C00904FF0000922E0009800F02B
:102E70008000802809D1AA1991B204EB09024244CA
:102E800090B2524600F032F80BE00E98504508D050
:102E9000AA1991B204EB0902424490B20E9A00F0D2
:102EA00025F800984006000E009009F1010000F09E
:102EB000FF09B9F1080FD9DB08F1080000F0FF089D
:102EC0000BF1010000F0FF0BBB45BDDB4FF000082C
:102ED000701CC6B204488068C088B042B1DC00BF34
:102EE000A0E70000260000203000002070B5044656
:102EF0000D461646002C09DB002D07DB094800882B
:102F0000A04203DD07484088A84200DC70BD2B4684
:102F100022462946204600F075FA304600F0A0FA15
:102F200000BFF3E72600002070B504460D48408836
:102F3000401E83B20B480088401E82B20021084622
:102F400000F060FA074800880649498800FB01F54F
:102F500002E0204600F084FA281EA5F10105F8D110
:102F600070BD0000260000201CB500200121034692
:102F70000246CDE90010FFF723FFA84908700020A2
:102F8000012103460A46CDE900100146FFF718FF6C
:102F9000A34908700020012103460246CDE9001034
:102FA00001460120FFF70CFF9E4908700020012117
:102FB00003460A46CDE900100846FFF701FF9A498B
:102FC000087000F0A5F9282000F045FACF2000F0A5
:102FD00042FA002000F044FA832000F041FA302049
:102FE00000F03EFAED2000F036FA642000F038FAE6
:102FF000032000F035FA122000F032FA812000F0B0
:103000002FFAE82000F027FA852000F029FA0120A5
:1030100000F026FA792000F023FACB2000F01BFA0A
:10302000392000F01DFA2C2000F01AFA002000F0E0
:1030300017FA342000F014FA022000F011FAF720F9
:1030400000F009FA202000F00BFAEA2000F003FA61
:10305000002000F005FA002000F002FAC02000F085
:10306000FAF9262000F0FCF9C12000F0F4F9112053
:1030700000F0F6F9C52000F0EEF9352000F0F0F987
:103080003E2000F0EDF9C72000F0E5F9BE2000F089
:10309000E7F9362000F0DFF96048007800F0E0F949
:1030A0003A2000F0D8F9552000F0DAF9B12000F00C
:1030B000D2F9002000F0D4F91B2000F0D1F9F22061
:1030C00000F0C9F9082000F0CBF9262000F0C3F980
:1030D000012000F0C5F9E02000F0BDF91F2000F04C
:1030E000BFF91A2000F0BCF9182000F0B9F90A2045
:1030F00000F0B6F90F2000F0B3F9062000F0B0F9A7
:10310000452000F0ADF9872000F0AAF9322000F048
:10311000A7F90A2000F0A4F9072000F0A1F9022085
:1031200000F09EF9072000F09BF9052000F098F9C7
:10313000002000F095F9E12000F08DF9002000F06A
:103140008FF9252000F08CF9272000F089F905205F
:1031500000F086F9102000F083F9092000F080F9D2
:103160003A2000F07DF9782000F07AF94D2000F047
:1031700077F9052000F074F9182000F071F90D209E
:1031800000F06EF9382000F06BF93A2000F068F991
:103190001F2000F065F92A2000F05DF9002000F002
:1031A0005FF9002000F05CF9002000F059F9EF20F1
:1031B00000F056F92B2000F04EF9002000F050F9F5
:1031C000002000F04DF9012000F04AF93F2000F006
:1031D00047F9B72000F03FF9072000F041F9B62089
:1031E00000F039F90A2000F03BF9822000F038F9AC
:1031F000272000F035F9002000F032F9112000F00E
:103200002AF96420FFF7B4FD292000F024F9642096
:10321000FFF7AEFD2C2000F01EF91CBD440000207D
:103220004500002046000020470000200FB47CB578
:1032300007A801903248019A0699FDF76BF8002023
:1032400001902F4C56E020780A280AD12D4840885A
:103250002D498968C98808442A4948800020088087
:103260003EE020780D283BD02078092809D1254858
:10327000018825488068808801EB8000214908800A
:103280002EE02148808880B21F4D00902D88ABB27F
:1032900022781C4D6D8829B21A4D2D8828B2FFF76F
:1032A000A7FD184800881849896889880844154985
:1032B00008801548007B98B1144800881249896835
:1032C0008988401A0F490988884209DA0D484088E0
:1032D0000D498968C98808440A4948800020088047
:1032E000641C0848408809494988884202DB00205C
:1032F0000449488020780028A5D17CBC5DF814FBE7
:103300003403002040000020300000202600002070
:1033100010B5012000F09FF83220FFF729FD10BD05
:1033200070B505460C4605480580448023462A466C
:103330002146284600F066F870BD000040000020DD
:1033400010B5044624480471362000F084F8224861
:10335000007930B101281AD002280DD003282CD1D1
:1033600020E01E48007800F07BF8F0201A49088021
:103370004FF4A070488021E01948007800F070F800
:10338000F020154908804FF4A070488016E01548D9
:10339000007800F065F84FF4A0700F490880F02025
:1033A00048800BE01048007800F05AF84FF4A07005
:1033B00009490880F020488000E000BF00BF0648AF
:1033C0004088401E83B204480088401E82B200211B
:1033D000084600F017F810BD260000204400002029
:1033E000460000204500002047000020014A1060F0
:1033F000516070473000002001498860704700002C
:10340000300000202DE9F04104460D4616461F46C7
:103410002A2000F020F8200A00F022F8E0B200F0A4
:103420001FF8300A00F01CF8F0B200F019F82B2059
:1034300000F011F8280A00F013F8E8B200F010F8D4
:10344000380A00F00DF8F8B200F00AF82C2000F06D
:1034500002F8BDE8F0814FF0C041088070470000DD
:10346000014908807047000000000860BCB0B14806
:1034700000684FF47A72B0FBF2F1481EB0F1807F21
:1034800000D31BE0481E4FF0E022506150170F227E
:10349000002804DB13071D0EA74B1D5406E013077D
:1034A0001E0EA64B00F00F052D1F5E5500BF00201D
:1034B0004FF0E02290610720106100BFFEF726FD6B
:1034C000FFF732FCFFF7B2F8FEF768FDFFF74CFD9F
:1034D0000120FFF735FF4FF6FF70FFF725FD322083
:1034E000FEF738FE9648FFF787FF4FF6FF71002082
:1034F000FFF77CFF05212820FFF712FF91A0FFF7BF
:1035000095FE9448FFF778FF4FF6FF710020FFF714
:103510006DFF002290A1934800F067F9002292A16C
:10352000904800F062F90A20FFF722FCFF218F4843
:10353000FDF744F84FF47A70FFF71AFC22208C490B
:10354000087078228B491EA8FDF706F87822894971
:1035500078316846FDF700F885491EA8FCF7F0FFB2
:1035600069461EA8FCF7ECFF81491EA8FCF7E8FF9E
:1035700000221EA97B4800F038F900227AA1794880
:1035800000F033F90A20FFF7F3FBFF217748FDF73E
:1035900015F80A20FFF7ECFB78211EA8FDF730F89C
:1035A0000024C5E0002CFCD10320734908700022E0
:1035B00072A16C4800F019F90A20FFF7D9FB7821B5
:1035C0007048FCF7FBFF694A6FA16E48FCF7B4FE38
:1035D000FF216648FCF7F2FF2D210A20FFF7A0FE2D
:1035E0006848FFF723FE4FF4FA60FFF7C1FB0220A3
:1035F00061490870002265A15A4800F0F6F80A20D7
:10360000FFF7B6FB78216348FCF7D8FF574A5EA165
:103610006048FCF791FEFF215448FCF7CFFF4121A1
:103620000A20FFF77DFE5B48FFF700FE4FF4FA60CB
:10363000FFF79EFB032050490870002256A149481D
:1036400000F0D3F80A20FFF793FB78215548FCF7E8
:10365000B5FF464A4CA15348FCF76EFEFF21434894
:10366000FCF7ACFF55210A20FFF75AFE4D48FFF743
:10367000DDFD4FF4FA60FFF77BFB01203E49087047
:10368000012249A1374800F0B0F80A20FFF770FB8B
:1036900078214848FCF792FF344A3BA14548FCF7A3
:1036A0004BFEFF213148FCF789FF69210A20FFF713
:1036B00037FE4048FFF7BAFD4FF4FA60FFF758FBBA
:1036C00002202D49087000223BA1264800F08DF809
:1036D0000A20FFF74DFB78213948FCF76FFF234A9A
:1036E00029A13748FCF728FEFF212048FCF766FF98
:1036F0006420FFF73DFB7D210A20FFF711FE3048D3
:10370000FFF794FD4FF4FA60FFF732FB80212D485C
:10371000FEF7F7FB6420FFF72BFB80212948FEF71B
:10372000F2FB40212748FEF7EEFB6420FFF720FB69
:1037300038E700005000002000E400E018ED00E051
:103740001C0000207777772E73746D3332726573A7
:103750002E7275001400002041542B434D47463D06
:1037600031000000004400400A0000003404002042
:1037700044020020983800080000002041542B47E4
:103780004D4D0A00CC0100202573000041542B4709
:103790004D520A006400002041542B434F50533FC8
:1037A0000A000000DC00002041542B43434C4B3FF7
:1037B000000000005401002041542B4342430A0002
:1037C000BC0200200000024000B9704708E0017808
:1037D0000A2902D001780D2901D120210170401C55
:1037E00001780029F3D100BFEFE770B506460C461B
:1037F000154604E014F8011B304600F009F8207863
:103800000028F7D11DB10D21304600F001F870BD40
:1038100070B504460D4600BF208800F080000028E7
:10382000FAD029462046FFF75CFA70BD10B5002992
:103830000AD00878002807D005487844FDF73AFEFA
:10384000002801D0002010BD0248784410BD0000BF
:103850009A2100009221000010B500290AD00878B2
:10386000002807D005487844FDF724FE002801D041
:10387000002010BD0248784410BD00008A210000DD
:10388000822100004FF04070E1EE100A7047FDF712
:1038900034BAFDF769BB000041542B43434C4B3D08
:1038A0000000000000000000000000000000000018
:1038B0000000000000000000000000000000000008
:1038C00000000000000000000000000000000000F8
:1038D00000000000000000000000000000000000E8
:1038E00000000000000000000000000000000000D8
:1038F00000000000000000000000000000000000C8
:1039000000000000000000000000000000000000B7
:1039100032302F30332F31322C32303A33303A3587
:10392000352B3033000000000000000000000000D4
:103930000000000000000000000000000000000087
:103940000000000000000000000000000000000077
:103950000000000000000000000000000000000067
:103960000000000000000000000000000000000057
:103970000000000000000000000000000000000047
:103980000000000000000000000000000000000037
:1039900000000000001010101010000010000000C7
:1039A000006C4848000000000000000000141428CB
:1039B0007C287C2850500000001038404038487067
:1039C00010100000002050200C70081408000000A7
:1039D000000000182020544834000000001010108F
:1039E0001000000000000000000808101010101067
:1039F00010080800002020101010101010202000C7
:103A000000107C10282800000000000000001010AA
:103A100010FE101010000000000000000000001850
:103A20001030200000000000007C000000000000BA
:103A30000000000000000030300000000004040816
:103A400008101020204000000038444444444444FE
:103A50003800000000301010101010107C00000022
:103A600000384404081020447C000000003844045E
:103A70001804044438000000000C141424447E048C
:103A80000E000000003C20203804044438000000F0
:103A9000001C20407844444438000000007C44046A
:103AA000080808101000000000384444384444441A
:103AB0003800000000384444443C04087000000012
:103AC000000000303000003030000000000000181E
:103AD000180000183020000000000C1060806010FA
:103AE0000C000000000000007C007C0000000000D2
:103AF0000000C02018041820C00000000000182496
:103B000004081000300000003844444C54544C4029
:103B1000443800000030102828287C44EE000000C3
:103B200000F8444478444444F8000000003C444019
:103B3000404040443800000000F0484444444448B9
:103B4000F000000000FC445070504044FC000000B5
:103B5000007E22283828202070000000003C4440CD
:103B6000404E44443800000000EE44447C44444449
:103B7000EE000000007C1010101010107C000000FF
:103B8000003C0808084848483000000000EE44485F
:103B900050704844E60000000070202020202424BB
:103BA0007C00000000EE6C6C54544444EE000000B5
:103BB00000EE64645454544CEC000000003844445B
:103BC0004444444438000000007824242438202051
:103BD000700000000038444444444444381C000051
:103BE00000F8444444784844E200000000344C406B
:103BF000380404645800000000FE921010101010E9
:103C00003800000000EE44444444444438000000BE
:103C100000EE4444282828101000000000EE444420
:103C2000545454542800000000C64428101028445E
:103C3000C600000000EE44282810101038000000D4
:103C4000007C4408101020447C0000000038202034
:103C500020202020202038000040202020101008A4
:103C60000808000000380808080808080808380094
:103C700000101028440000000000000000000000B8
:103C800000000000000000FE00100800000000001E
:103C90000000000000000038443C44443E000000A6
:103CA00000C0405864444444F80000000000003C58
:103CB0004440404438000000000C04344C44444468
:103CC0003E00000000000038447C40403C00000002
:103CD000001C207C202020207C00000000000036FA
:103CE0004C4444443C04380000C0405864444444BC
:103CF000EE00000000100070101010107C0000009A
:103D000000100078080808080808700000C0405C2F
:103D100048705048DC0000000030101010101010E7
:103D20007C000000000000E854545454FE000000E1
:103D3000000000D864444444EE0000000000003855
:103D40004444444438000000000000D86444444423
:103D50007840E000000000364C4444443C040E002F
:103D60000000006C302020207C0000000000003C9F
:103D700044380444780000000000207C20202022E9
:103D80001C000000000000CC4444444C36000000FD
:103D9000000000EE4444282810000000000000EE5F
:103DA0004454545428000000000000CC48303048EF
:103DB000CC000000000000EE442428181010780009
:103DC0000000007C481020447C0000000008101017
:103DD00010102010101008000010101010101010FB
:103DE00010100000002010101010081010102000FB
:103DF0000000000000245800000000000000000047
:103E000000000000000000000000000000000000B2
:103E100000000000000000000000000000000000A2
:103E20000000000000000000000000000000000092
:103E30000000000000000000000000000000000082
:103E4000000000000000000000000380000380006C
:103E500003800003800003800003800003800003D0
:103E6000800003800001000001000000000000004D
:103E7000000380000380000000000000000000003C
:103E80000000000000000000000000000000000032
:103E900000000000000E70000E70000E7000042084
:103EA00000042000042000042000000000000000A6
:103EB0000000000000000000000000000000000002
:103EC00000000000000000000000000000000000F2
:103ED0000000000000000000000006600006600016
:103EE0000660000660000660003FF8003FF800062C
:103EF00060000CC0003FF8003FF8000CC0000CC090
:103F0000000CC0000CC0000CC0000000000000004D
:103F100000000000000000000000000000000001A0
:103F2000800001800007B0000FF0001870001870CA
:103F3000001C00000F800007E00000F000183000B7
:103F40001C30001C70001FE0001BC000018000013D
:103F500080000180000180000000000000000000DF
:103F6000000000000000000000000780000FC000FB
:103F70001CE0001860001860001CE0000FF800074B
:103F8000E0001FF000073800061800061800073888
:103F90000003F00001E0000000000000000000004D
:103FA0000000000000000000000000000000000011
:103FB000000000000000000003F00007F0000C60AB
:103FC000000C00000C00000600000700000F9C0021
:103FD0001DFC0018F0001870000FFC0007DC00004A
:103FE00000000000000000000000000000000000D1
:103FF000000000000000000000000000000380003E
:1040000003800003800001000001000001000001A6
:1040100000000000000000000000000000000000A0
:104020000000000000000000000000000000000090
:104030000000000000000000000000000000000080
:10404000000000180000380000700000F00000E0E0
:104050000000E00001C00001C00001C00001C0007C
:1040600001C00001C00000E00000E000007000009E
:104070007000003800001800000000000000000080
:10408000000000000000000000001800001C0000FC
:104090000E00000E00000700000700000380000370
:1040A000800003800003800003800003800007007D
:1040B000000700000F00000E00001C0000180000A8
:1040C00000000000000000000000000000000000F0
:1040D00000000180000180000180001DB8001FF871
:1040E0000007E00003C00003C00006600006600097
:1040F00000000000000000000000000000000000C0
:1041000000000000000000000000000000000000AF
:10411000000000000000000000000000000000009F
:104120000180000180000180000180000180003FCB
:10413000FC003FFC00018000018000018000018044
:1041400000018000000000000000000000000000EE
:10415000000000000000000000000000000000005F
:10416000000000000000000000000000000000004F
:10417000000000000000000000000000000000003F
:1041800000000000000000E00000C00001C00001CD
:104190008000018000030000030000000000000018
:1041A000000000000000000000000000000000000F
:1041B0000000000000000000000000000000001FE0
:1041C000F8001FF8000000000000000000000000E0
:1041D00000000000000000000000000000000000DF
:1041E00000000000000000000000000000000000CF
:1041F00000000000000000000000000000000000BF
:1042000000000000000000000000000000000000AE
:1042100000000000000003C00003C00003C0000055
:10422000000000000000000000000000000000008E
:1042300000000000001800001800003800003000E6
:1042400000700000600000600000C00000C00001BD
:10425000800001800003000003000006000006004B
:10426000000E00000C00001C0000180000180000E8
:10427000000000000000000000000000000000003E
:10428000000003C00007E0000C30000C30001818DC
:10429000001818001818001818001818001818002E
:1042A0001818000C30000C300007E00003C00000BC
:1042B00000000000000000000000000000000000FE
:1042C00000000000000000000000008000078000E7
:1042D0001F80001D8000018000018000018000011E
:1042E00080000180000180000180000180000180C9
:1042F000001FF8001FF80000000000000000000090
:1043000000000000000000000000000000000000AD
:10431000000007C0001FF0003830003018003018CF
:104320000000180000300000600001C000038000A1
:104330000600000C00001800003FF8003FF80000E5
:10434000000000000000000000000000000000006D
:104350000000000000000000000003C0000FE000AB
:104360000C700000300000300000600003C000034B
:10437000E000007000001800001800001800183855
:10438000001FF0000FC0000000000000000000004F
:10439000000000000000000000000000000000001D
:1043A000000000E00001E00001E0000360000660A2
:1043B000000660000C60000C6000186000306000B7
:1043C0003FF8003FF80000600003F80003F8000029
:1043D00000000000000000000000000000000000DD
:1043E000000000000000000000001FF0001FF000AF
:1043F0001800001800001800001BC0001FF0001C6F
:1044000030000018000018000018000018003030BC
:10441000003FF0000FC0000000000000000000009E
:10442000000000000000000000000000000000008C
:10443000000000F80003F8000700000E00000C0068
:10444000001800001BC0001FF0001C3000181800EE
:104450001818001818000C38000FF00003E00000D6
:10446000000000000000000000000000000000004C
:10447000000000000000000000001FF8001FF8000E
:1044800018180018380000300000300000700000DC
:10449000600000600000E00000C00000C00001C03B
:1044A000000180000180000000000000000000000A
:1044B00000000000000000000000000000000000FC
:1044C000000007E0000FF0001C3800181800181852
:1044D000000C300007E00007E0000C300018180066
:1044E0001818001818001C38000FF00007E0000032
:1044F00000000000000000000000000000000000BC
:104500000000000000000000000007C0000FF000E5
:104510001C30001818001818001818000C38000F6C
:10452000F80003D80000180000300000700000E020
:10453000001FC0001F00000000000000000000007D
:10454000000000000000000000000000000000006B
:10455000000000000000000000000000000003C098
:104560000003C00003C000000000000000000000C5
:1045700000000000000003C00003C00003C00000F2
:10458000000000000000000000000000000000002B
:10459000000000000000000000000000000000001B
:1045A00000000000000000F00000F00000F000003B
:1045B000000000000000000000000000E00001C05A
:1045C00000018000018000030000020000000000E4
:1045D00000000000000000000000000000000000DB
:1045E0000000000000000000001C00003C0000F083
:1045F0000003C0000F00003C0000F000003C000081
:104600000F000003C00000F000003C00001C000090
:10461000000000000000000000000000000000009A
:10462000000000000000000000000000000000008A
:104630000000000000000000007FFC007FFC000084
:1046400000000000007FFC007FFC00000000000074
:10465000000000000000000000000000000000005A
:10466000000000000000000000000000000000004A
:1046700000000000000000007000007800001E0034
:104680000007800001E000007800001E00007800B4
:1046900001E0000780001E000078000070000000AC
:1046A000000000000000000000000000000000000A
:1046B0000000000000000000000000000007C00033
:1046C0000FE0001870001830001830000070000073
:1046D000E00003C0000380000300000000000000B1
:1046E00000070000070000000000000000000000BC
:1046F00000000000000000000000000000000000BA
:10470000000003E00007F0000E38000C18001878D5
:104710000018F80019D80019980019980019980085
:1047200018F8001878001800000C00000E18000798
:10473000F80003E00000000000000000000000009E
:10474000000000000000000000000000001F8000CA
:104750001FC00001C00003600003600006300006B7
:1047600030000C30000FF8001FF800180C00300C5F
:1047700000FC7F00FC7F0000000000000000000043
:104780000000000000000000000000000000000029
:1047900000000000007FE0007FF0001838001818CB
:1047A000001818001838001FF0001FF800181C002F
:1047B000180C00180C00180C007FF8007FF00000A7
:1047C00000000000000000000000000000000000E9
:1047D0000000000000000000000000000003EC00EA
:1047E0000FFC001C1C00180C00300C0030000030C6
:1047F0000000300000300000300000180C001C1CCD
:10480000000FF80003F000000000000000000000AE
:104810000000000000000000000000000000000098
:1048200000000000007FC0007FF00018380018185A
:1048300000180C00180C00180C00180C00180C00C4
:10484000180C001818001838007FF0007FE00000F6
:104850000000000000000000000000000000000058
:10486000000000000000000000000000007FF800D1
:104870007FF8001818001818001998001980001FF8
:1048800080001F800019800019980018180018185F
:10489000007FF8007FF8000000000000000000002A
:1048A0000000000000000000000000000000000008
:1048B00000000000003FFC003FFC000C0C000C0C52
:1048C000000CCC000CC0000FC0000FC0000CC000DA
:1048D0000CC0000C00000C00003FC0003FC00000F6
:1048E00000000000000000000000000000000000C8
:1048F0000000000000000000000000000003EC00C9
:104900000FFC001C1C00180C00300C0030000030A4
:10491000000030FE0030FE00300C00380C001C1C83
:10492000000FFC0003F00000000000000000000089
:104930000000000000000000000000000000000077
:1049400000000000007E7E007E7E0018180018180F
:10495000001818001818001FF8001FF80018180099
:104960001818001818001818007E7E007E7E0000BF
:104970000000000000000000000000000000000037
:10498000000000000000000000000000001FF80010
:104990001FF80001800001800001800001800001FB
:1049A0008000018000018000018000018000018002
:1049B000001FF8001FF800000000000000000000C9
:1049C00000000000000000000000000000000000E7
:1049D000000000000007FE0007FE0000300000306D
:1049E0000000300000300000300030300030300077
:1049F0003030003030003060003FE0000F800000B9
:104A000000000000000000000000000000000000A6
:104A1000000000000000000000000000007F3E00D9
:104A20007F3E0018300018600018C0001980001B7D
:104A300080001FC0001CE0001870001830001838FB
:104A4000007F1F007F1F000000000000000000002A
:104A50000000000000000000000000000000000056
:104A600000000000007F80007F80000C00000C0030
:104A7000000C00000C00000C00000C00000C0C00EE
:104A80000C0C000C0C000C0C007FFC007FFC0000E8
:104A90000000000000000000000000000000000016
:104AA00000000000000000000000000000F00F0007
:104AB000F81F00381C003C3C003C3C00366C0036C3
:104AC0006C0033CC0033CC00318C00300C00300C47
:104AD00000FE7F00FE7F00000000000000000000DC
:104AE00000000000000000000000000000000000C6
:104AF000000000000078FE0078FE001C18001E1860
:104B0000001F18001B18001B980019D80018D800A7
:104B100018F8001878001838007F18007F18000077
:104B20000000000000000000000000000000000085
:104B30000000000000000000000000000003C000B2
:104B40000FF0001C3800181800381C00300C003022
:104B50000C00300C00300C00381C001818001C38F9
:104B6000000FF00003C00000000000000000000083
:104B70000000000000000000000000000000000035
:104B800000000000003FF0003FF8000C1C000C0C7F
:104B9000000C0C000C0C000C18000FF8000FE000CB
:104BA0000C00000C00000C00003FC0003FC00000E3
:104BB00000000000000000000000000000000000F5
:104BC0000000000000000000000000000003C00022
:104BD0000FF0001C3800181800381C00300C003092
:104BE0000C00300C00300C00381C001818001C3869
:104BF000000FF00007C00007CC000FFC000C3800CD
:104C000000000000000000000000000000000000A4
:104C100000000000007FE0007FF000183800181846
:104C2000001818001838001FF0001FC00018E0001E
:104C30001870001830001838007F1E007F0E00002A
:104C40000000000000000000000000000000000064
:104C50000000000000000000000000000007D80075
:104C60000FF8001C38001818001818001E00000F5C
:104C7000C00003F0000078001818001818001C3855
:104C8000001FF0001BE0000000000000000000001A
:104C90000000000000000000000000000000000014
:104CA00000000000003FFC003FFC00318C00318C14
:104CB00000318C00318C00018000018000018000F7
:104CC0000180000180000180000FF0000FF0000063
:104CD00000000000000000000000000000000000D4
:104CE000000000000000000000000000007E7E00C8
:104CF0007E7E0018180018180018180018180018E0
:104D000018001818001818001818001818000C308F
:104D1000000FF00003C000000000000000000000D1
:104D20000000000000000000000000000000000083
:104D300000000000007F7F007F7F00180C000C182F
:104D4000000C18000C18000630000630000360004C
:104D500003600003600001C00001C000008000008B
:104D60000000000000000000000000000000000043
:104D700000000000000000000000000000FE3F8076
:104D8000FE3F8030060030060030860019CC001946
:104D9000CC001B6C001B6C001E7C000E38000E3813
:104DA000000C18000C1800000000000000000000BB
:104DB00000000000000000000000000000000000F3
:104DC00000000000007E7E007E7E001818000C307F
:104DD0000006600003C00001800001800003C000E5
:104DE0000660000C30001818007E7E007E7E0000F9
:104DF00000000000000000000000000000000000B3
:104E0000000000000000000000000000007C7E00A8
:104E10007C7E001818000C3000066000066000035D
:104E2000C00001800001800001800001800001803D
:104E3000000FF0000FF00000000000000000000074
:104E40000000000000000000000000000000000062
:104E500000000000001FF8001FF8001818001830AC
:104E60000018600018C00001800003000006180050
:104E70000C18001818003018003FF8003FF8000028
:104E80000000000000000000000000000000000022
:104E90000000000000000000000001F00001F00030
:104EA000018000018000018000018000018000017C
:104EB00080000180000180000180000180000180ED
:104EC0000001800001800001800001F00001F0007D
:104ED00000000000000000000000000018000018A2
:104EE00000001C00000C00000E0000060000060080
:104EF0000003000003000001800001800000C000EA
:104F000000C0000060000060000070000030000081
:104F10003800001800001800000000000000000029
:104F2000000000000000000000000F80000F800063
:104F300001800001800001800001800001800001EB
:104F4000800001800001800001800001800001805C
:104F5000000180000180000180000F80000F8000B0
:104F60000000000000000000000000000000000041
:104F7000800001C00003E0000770000630000C183C
:104F800000180C00100400000000000000000000E9
:104F90000000000000000000000000000000000011
:104FA0000000000000000000000000000000000001
:104FB00000000000000000000000000000000000F1
:104FC00000000000000000000000000000000000E1
:104FD00000000000000000000000000000000000D1
:104FE00000000000000000000000000000000000C1
:104FF000000000000000FFFF00FFFF0000000003B2
:10500000000003800000E0000060000000000000DD
:105010000000000000000000000000000000000090
:105020000000000000000000000000000000000080
:105030000000000000000000000000000000000070
:105040000000000000000000000000000000000060
:105050000000000000000FC0001FE0000030000052
:10506000300007F0001FF0003830003030003070A2
:10507000001FFC000FBC000000000000000000004A
:105080000000000000000000000000000000000020
:1050900000007800007800001800001800001BE0F5
:1050A000001FF8001C1800180C00180C00180C0049
:1050B000180C00180C001C18007FF8007BE00000A2
:1050C00000000000000000000000000000000000E0
:1050D00000000000000000000000000000000000D0
:1050E00000000000000003EC000FFC001C1C003856
:1050F0000C00300C00300000300000380C001C1C8C
:10510000000FF80003F000000000000000000000A5
:10511000000000000000000000000000000000008F
:10512000000000780000780000180000180007D880
:10513000001FF80018380030180030180030180030
:105140003018003018001838001FFE0007DE00007D
:10515000000000000000000000000000000000004F
:10516000000000000000000000000000000000003F
:1051700000000000000007E0001FF80018180030D1
:105180000C003FFC003FFC00300000300000180C19
:10519000001FFC0007F000000000000000000000FD
:1051A00000000000000000000000000000000000FF
:1051B000000001FC0003FC000600000600003FF8B0
:1051C000003FF80006000006000006000006000090
:1051D0000600000600000600003FF0003FF000005F
:1051E00000000000000000000000000000000000BF
:1051F00000000000000000000000000000000000AF
:1052000000000000000007DE001FFE00183800301C
:105210001800301800301800301800301800183806
:10522000001FF80007D80000180000180000380020
:105230000FF0000FC00000000000000000000000A0
:1052400000007800007800001800001800001BE043
:10525000001FF0001C38001818001818001818005B
:105260001818001818001818007E7E007E7E0000B6
:10527000000000000000000000000000000000002E
:10528000000000000000000000000180000180001C
:105290000000000000001F80001F8000018000014E
:1052A00080000180000180000180000180000180F9
:1052B000003FFC003FFC0000000000000000000078
:1052C00000000000000000000000000000000000DE
:1052D000000000C00000C0000000000000001FF03F
:1052E000001FF000003000003000003000003000EF
:1052F00000300000300000300000300000300000BE
:1053000030000030000070001FE0001F800000002F
:10531000000000000000000000003C00003C000015
:105320000C00000C00000CF8000CF8000CC0000D84
:1053300080000F80000F00000F80000DC0000CE007
:10534000003C7C003C7C00000000000000000000ED
:10535000000000000000000000000000000000004D
:1053600000001F80001F800001800001800001807C
:1053700000018000018000018000018000018000A8
:105380000180000180000180003FFC003FFC000024
:10539000000000000000000000000000000000000D
:1053A00000000000000000000000000000000000FD
:1053B000000000000000F77800FFFC0039CC00314D
:1053C0008C00318C00318C00318C00318C00318CA0
:1053D00000FDEF00FDEF00000000000000000000F5
:1053E00000000000000000000000000000000000BD
:1053F00000000000000000000000000000007BE052
:10540000007FF0001C380018180018180018180049
:105410001818001818001818007E7E007E7E000004
:10542000000000000000000000000000000000007C
:10543000000000000000000000000000000000006C
:1054400000000000000003C0000FF0001C3800380E
:105450001C00300C00300C00300C00381C001C38D4
:10546000000FF00003C0000000000000000000007A
:10547000000000000000000000000000000000002C
:1054800000000000000000000000000000007BE0C1
:10549000007FF8001C1800180C00180C00180C00F5
:1054A000180C00180C001C18001FF8001BE0001856
:1054B00000001800001800007F00007F00000000BE
:1054C00000000000000000000000000000000000DC
:1054D00000000000000007DE001FFE00183800304A
:1054E0001800301800301800301800301800183834
:1054F000001FF80007D8000018000018000018006E
:1055000000FE0000FE00000000000000000000009F
:1055100000000000000000000000000000003E78D5
:10552000003EFC0007CC000700000600000600005B
:105530000600000600000600003FF0003FF00000FB
:10554000000000000000000000000000000000005B
:10555000000000000000000000000000000000004B
:1055600000000000000007F8000FF80018180018ED
:1055700018001F80000FF00000F8001818001838FD
:10558000001FF0001FE0000000000000000000000D
:10559000000000000000000000000000000000000B
:1055A00000000C00000C00000C00000C00003FF09C
:1055B000003FF0000C00000C00000C00000C00008C
:1055C0000C00000C00000C1C0007FC0003F00000A5
:1055D00000000000000000000000000000000000CB
:1055E00000000000000000000000000000000000BB
:1055F0000000000000007878007878001818001883
:105600001800181800181800181800181800183872
:10561000000FFE0007DE0000000000000000000098
:10562000000000000000000000000000000000007A
:1056300000000000000000000000000000007C3EB0
:10564000007C3E001818001818000C30000C3000C8
:1056500006600006600007E00003C00003C0000011
:10566000000000000000000000000000000000003A
:10567000000000000000000000000000000000002A
:10568000000000000000783C00783C003118003336
:1056900098003398001AB0001EF0001EF0001C6045
:1056A000000C60000C600000000000000000000022
:1056B00000000000000000000000000000000000EA
:1056C00000000000000000000000000000003E7C20
:1056D000003E7C000C300006600003C0000180002A
:1056E00003C0000660000C30003E7C003E7C0000E1
:1056F00000000000000000000000000000000000AA
:105700000000000000000000000000000000000099
:105710000000000000007E1F007E1F00180C000C1F
:1057200018000C180006300006300003600003E08B
:105730000001C00000C000018000018000030000E3
:105740003FC0003FC000000000000000000000005B
:1057500000000000000000000000000000001FF832
:10576000001FF80018300018600000C00001800021
:105770000300000618000C18001FF8001FF80000B6
:105780000000000000000000000000000000000019
:105790000000000000000000000000E00001E00048
:1057A0000180000180000180000180000180000173
:1057B000800003800007000003800001800001805A
:1057C0000001800001800001800001E00000E00095
:1057D00000000000000000000000000000000000C9
:1057E0000000018000018000018000018000018034
:1057F0000001800001800001800001800001800024
:105800000180000180000180000180000180000112
:105810008000018000018000000000000000000006
:1058200000000000000000000000070000078000EA
:1058300001800001800001800001800001800001E2
:10584000800001C00000E00001C000018000018074
:105850000001800001800001800007800007000037
:105860000000000000000000000000000000000038
:105870000000000000000000000000000000000028
:10588000000000000E00001F18003BB80031F000BF
:1058900000E0000000000000000000000000000028
:1058A00000000000000000000000000000000000F8
:1058B00000000000040000080000000000000002DA
:1058C00000010000100000000000000000000000C7
:1058D0003031323334353637383941424344454626
:1058E0004030580030313233343536373839616220
:1058F0006364656640307800303132333435363792
:1059000038396162636465667870003031323334EF
:105910003536373839414243444546585000000037
:1059200002400000000000A0000000000540000050
:10593000000000C8000000000C4000000000409C77
:1059400000000000194000000020BCBE0000000064
:1059500034400000BFC91B8E00000004B5400000A9
:10596000504BCFD06607E2CF010000006C41000031
:105970003E8251AADFEEA73401000000D9420000A8
:10598000DCB5A0E23A301F97FFFFFFFFB4450000EF
:10599000FD25A0C8E9A3C14FFFFFFFFFFF3F0000A7
:1059A0000000008000000000FF3F000000000080B9
:1059B00000000000005B0008000000206400000000
:1059C000C4010008645B000864000020AC0B000008
:1059D000E00100081C00000043000000F8FFFFFF8A
:1059E0000C0000000E0000000F0000002E00000060
:1059F0001001000043000000F8FFFFFF004040409E
:105A00004040404040404141414141404040404091
:105A1000404040404040404040404040400502023D
:105A200002020202020202020202020202202020FC
:105A30002020202020202002020202020202909058
:105A40009090909010101010101010101010101056
:105A500010101010101010100202020202028888AA
:105A600088888888080808080808080808080808B6
:105A7000080808080808080802020202400000009E
:105A80000000000000000000000000000000000016
:105A90000000000000000000000000000000000006
:105AA00000000000000000000000000000000000F6
:105AB00000000000000000000000000000000000E6
:105AC00000000000000000000000000000000000D6
:105AD00000000000000000000000000000000000C6
:105AE00000000000000000000000000000000000B6
:105AF00000000000000000000000000000000000A6
:105B0000000000000001020304010203040607086C
:105B1000090000008839000807000C00FC3D00085F
:105B2000110018000000F000400100010100000019
:105B3000E0FF000000000000140000200100000051
:105B40000000000000000000000000000000000055
:105B5000007A030A000000000000000001020304B4
:045B60000607080923
:040000050800018965
:00000001FF
